:020000040000FA
:1000000007EF00F0FFFFFFFF5D825EED19F059EF93
:1000100018F0070E926E9368180E946E956A966AA1
:10002000896A8A688B6A8C6A8D6A0C0EC16EBE0EF4
:10003000C06EF19EBA6AD56A300ECD6ECA6ACF6ABA
:10004000CE6A9D80F28CF290F286F29E400E116E86
:10005000420E126E0F0E136E146ACBEC1AF0060EDF
:10006000546E130E536EAE0EE82EFED7532EFCD7F1
:10007000542EFAD7CFEC19F0B8EC1CF0010EDAECE4
:100080001CF0000E19EC1DF00001C06F010E19EC00
:100090001DF05C6E020E19EC1DF00001C36F030E23
:1000A00019EC1DF0536E533002E3558001D055908A
:1000B000600E19EC1DF00001B96F610E19EC1DF016
:1000C0000001B86F620E19EC1DF00001BA6F630EEB
:1000D00019EC1DF00001BE6FBE5102E1520ED36F4C
:1000E000BE0502E1920ED36F020EBE1902E1D20EDE
:1000F000D36F040EE4EC18F006C0CCF007C0CDF0CE
:1001000008C0CEF009C0CFF0080EE4EC18F006C02D
:1001100094F007C095F008C096F009C097F06C0EF7
:10012000E4EC18F006C090F007C091F008C092F01F
:1001300009C093F0700EE4EC18F006C08CF007C014
:100140008DF008C08EF009C08FF0100E1FEC1CF06F
:10015000120E1FEC1CF00C0E1FEC1CF006C0ACF0D5
:1001600007C0ADF09FEC08F00EEC08F066EC1BF059
:10017000C5EC17F0CFEC08F0F7EC1CF088EC08F0B9
:100180009BEC1AF0C2EC08F053EC1CF0086A030E6A
:10019000076E0A6AFC0E096E6BEC1CF0086A950E7D
:1001A000E3EC08F06BEC1CF0086A0F0EE3EC08F0CF
:1001B0006BEC1CF0086A100E076E4C0E0001B9259E
:1001C000AAEC08F06BEC1CF0086A110E076E6C0EBE
:1001D0000001B825AAEC08F06BEC1CF0086A120EBE
:1001E0002EEC08F06BEC1CF0086A130E2EEC08F0F5
:1001F0006BEC1CF0086A140E2EEC08F06BEC1CF093
:10020000086A150E2EEC08F06BEC1CF0086A160E4E
:100210002EEC08F06BEC1CF0086A170E2EEC08F0C0
:100220006BEC1CF0086AB70E076ED3C009F00A6ABF
:100230006BEC1CF0086AB10E076E0A6AA00E096E1C
:100240006BEC1CF05FEF05F0040E0001D71902E122
:10025000F29E02D0F28ECD805CEC08F065EC08F0E6
:10026000C0C0D6F055AE02D0558C01D0559C41ECA3
:1002700008F08150CF0BCD0A20E1060E546E130E0C
:10028000536EAE0EE82EFED7532EFCD7542EFAD75F
:100290008150CF0BCD0AFCE0060E546E130E536E48
:1002A000AE0EE82EFED7532EFCD7542EFAD70001FF
:1002B000C32B020EC36501D0C36B8150CF0B8F0AD5
:1002C0001FE1060E546E130E536EAE0EE82EFED7CF
:1002D000532EFCD7542EFAD755BE02D0558E01D0DE
:1002E000559E8150CF0B8F0AFCE0060E546E130E04
:1002F000536EAE0EE82EFED7532EFCD7542EFAD7EF
:100300008150CF0B4F0A2BE1060E546E130E536E25
:10031000AE0EE82EFED7532EFCD7542EFAD723EC80
:1003200008F0CBEC1BF055B002D0558001D05590B1
:100330008150CF0B4F0AFCE0060E546E130E536E25
:10034000AE0EE82EFED7532EFCD7542EFAD7CCECA7
:1003500008F006EC1AF0C5EC08F053EC1CF08150E4
:10036000CF0BCB0A1FE1060E546E130E536EAE0E6A
:10037000E82EFED7532EFCD7542EFAD78150CF0B40
:10038000CB0AFCE0060E546E130E536EAE0EE82E32
:10039000FED7532EFCD7542EFAD755B202D0558231
:1003A00001D055920001B7510AE0B751800A7F0F82
:1003B00003E3D2EC08F003D0B7BFD6EC08F0040E8C
:1003C000D71906E1C5EC17F00E6AD45198EC12F07B
:1003D0000EEC16F0C06F98EC19F05C6EBCD0E00E1D
:1003E0000001846F670E856F350E866F876B806B9B
:1003F000090E816F3D0E826F836B010ED56F55B074
:1004000002D0200EA6D0240EA4D0C00E0001846F0E
:10041000CF0E856F6A0E866F876B806BDD0E816FE6
:100420006D0E826F836B020ED56F55B002D0280E11
:1004300090D02C0E8ED0200E0001846F1D0E856F83
:100440009A0E866F876B700E806FE00E816F9A0E2A
:10045000826F836B040ED56F55B002D0300E79D009
:10046000340E77D0800E0001846F9F0E856FD50EFD
:10047000866F876BB00E806FF60E816FDA0E826F1B
:10048000836B080ED56F55B002D0380E62D03C0E8B
:1004900060D0800E0001846FA80E856F120E866FEB
:1004A000010E876FC00E806F380E816F150E826F40
:1004B000010E836F100ED56F55B002D0400E49D09B
:1004C000440E47D0400E0001846F6F0E856F400EC2
:1004D000866F010E876F100E806F4D0E816F470E75
:1004E000826F010E836F200ED56F55B002D0480E7B
:1004F00030D04C0E2ED0900E0001846FCA0E856F46
:100500007B0E866F010E876F300E806F510E816FEC
:100510007D0E826F010E836F400ED56F55B002D0F5
:10052000500E17D0540E15D00001846B3F0E856F0E
:10053000AB0E866F010E876FA00E806F2F0E816F3E
:10054000C50E826F010E836F800ED56F580E55B0A9
:100550005C0EBF6F14D05C5001E141D7010A01E18C
:1005600054D7030A01E167D7010A01E17BD7070AE3
:1005700090E0010AA7E0030ABEE0010AD5E0D5C079
:100580008CFF040E0001D7190CE0BD515C1809E185
:10059000010E55A0000E536E010E55AA000E531AFF
:1005A0000DE0BF51E4EC18F006C0C8F007C0C9F078
:1005B00008C0CAF009C0CBF05CEC08F00001BD51E6
:1005C0005C1815E0010E5C6402D0C36F01D0C36BF0
:1005D0005CC004F0010E94EC1CF009D0E2EC07F0D2
:1005E0000DD0D1EC07F00AD0F3EC07F007D00001F2
:1005F000C351F4E0010AF5E0030AF6E0C35102E159
:100600008B8C01D08B9CC30502E18B8E01D08B9E1D
:10061000020EC31902E1898A01D0899A000E38ECD2
:100620001AF00BC0B0F00CC0B1F0B0C004F0B1C013
:1006300005F0C8EC08F041EC1BF004C0B0F005C0B8
:10064000B1F00001B15103E1530EB05D03E3B16BB2
:10065000520EB06F4BEC08F010EC18F055B241D0D0
:10066000030E31EC15F08BEC1BF00001D70509E10E
:10067000C451C827C551C923C651CA23C751CB236A
:10068000D76BC851805DC9518159CA518259CB512C
:10069000835908E280C0C8F081C0C9F082C0CAF0A6
:1006A00083C0CBF0020ED71909E1C451C85FC55110
:1006B000C95BC651CA5BC751CB5BD76B8451C85D60
:1006C0008551C9598651CA598751CB5901E33DD14A
:1006D00084C0C8F085C0C9F086C0CAF087C0CBF01E
:1006E00034D1DAEC08F0F7EC1CF0FC0E406E7F0E13
:1006F000416E9BEC1AF029D104EC1DF00001BA0503
:1007000004E1220EBC6F1A0E03D01A0EBC6F220E2B
:10071000BB6FA9EC07F0BCC040F0E7EC08F0C8ECF8
:1007200007F0BBC040F0E7EC08F0DDEC08F006ECA9
:100730001AF0CFEC08F0F7EC1CF0AFEC08F09BECF3
:100740001AF0C2EC08F053EC1CF039EC1CF0D2D0DB
:1007500097EC13F0B4EC08F020EC13F0A5EC08F0E3
:100760001A0E046E000EF7EC1CF0F30E406E7F0EB6
:10077000416E9BEC1AF00001AA51AB1124E0AAC013
:1007800004F0ABC005F0BEEC08F041EC1BF033EC1C
:1007900008F009EC14F083EC08F09BEC1AF0AAC006
:1007A00004F0ABC005F0076A0A0E066EACEC1BF055
:1007B0003AEC08F009EC14F0AF0E406E7F0E416E7B
:1007C0009BEC1AF013D0B9EC08F00EEC12F01A0EF4
:1007D000046E110EF7EC1CF0B9EC08F00EEC12F000
:1007E000AD0E406E7F0E416E9BEC1AF01A0E046E39
:1007F0002A0EF7EC1CF0010E2BEC1DF0F00E406EF3
:100800007F0E416E9BEC1AF076EC08F041EC1BF089
:1008100033EC08F009EC14F083EC08F09BEC1AF0D0
:100820006EEC08F0ACEC1BF03AEC08F009EC14F0BC
:10083000E50E406E7F0E416E9BEC1AF039EC1CF019
:10084000020E38EC1AF00BC0A6F00CC0A7F0A6C040
:1008500004F0A7C005F0C8EC08F041EC1BF004C0A0
:10086000A6F005C0A7F00001A75103E1530EA65D55
:1008700003E3A76B530EA66F250E386EA6C039F0A2
:10088000A7C03AF0020E3B6E000E10EC18F0010EFD
:1008900038EC1AF00BC0A8F00CC0A9F0A8C004F006
:1008A000A9C005F0C8EC08F041EC1BF004C0A8F0AA
:1008B00005C0A9F00001A95103E1530EA85D03E3AF
:1008C000A96B530EA86F2B0E386EA8C039F0A9C0C3
:1008D0003AF0010E3B6E000E10EC18F0030E546E51
:1008E000080E536E770EE82EFED7532EFCD7542EEB
:1008F000FAD700F08150CF0BC30A01E129D79FEC52
:1009000008F027DBBCC040F0E7EC08F041DBBBC0DF
:1009100040F0E7EC08F039EC1CF004EC1DF0CFECF3
:1009200008F0F7EC1CF0AFEC08F09BEC1AF0DDECF3
:1009300008F006EC1AF0C2EC08F053EC1CF06EDB89
:1009400066EC1BF0A8DB10EC18F08150CF0BC30A4B
:1009500001E1D2D6010E55AA000EE5DB07E0000E3C
:1009600055B0010E046E030E94EC1CF0040E000151
:10097000D71917E0D651C01914E1BD515C1811E127
:10098000C251C3190EE1010E55AA000ECCDB09E1DC
:10099000010E55A8000E536E010E55A6000E531AF7
:1009A00014E0FADB06EC1AF0E0EC08F0F7EC1CF0CF
:1009B000AFDB9BEC1AF0E9DB53EC1CF039EC1CF0DC
:1009C00022EC17F00EEC16F0C06F040ED71917E0EA
:1009D0008851C81914E18951C91911E18A51CA19FC
:1009E0000EE18B51CB190BE1C251C31908E1BD5186
:1009F0005C1805E1010E55AA000E8FDB10E0C8C09F
:100A000042F0C9C043F0CAC044F0CBC045F0E8ECA6
:100A100014F000019EDABCC040F0E7EC08F0040ED0
:100A20000001D7190BE0C251C31908E1BD515C1890
:100A300005E1010E55AA000E70DB05E0A9DABBC086
:100A400040F0E7EC08F000018851C8190FE1895126
:100A5000C9190CE18A51CA1909E18B51CB1906E178
:100A6000C251C31903E1BD515C1804E0A44BA52B8E
:100A7000CE6ACF6AA451A51110E055A40ED0C3C010
:100A800004F0020E94EC1CF0DEDACBEC1BF000015B
:100A9000A46BA56B5594CE6ACF6AD76B22EC17F086
:100AA0007BDB06EC1AF08CDBF7EC1CF031DB9BEC0B
:100AB0001AF06BDB53EC1CF0B1DA66EC1BF055AEB0
:100AC00024EF01F0B8EC1CF00EEC16F0C06F040E31
:100AD000D76F3BD2C15102E1B8EC1CF0F6DA55AE4B
:100AE00002D0558C01D0559CCCDA55A602D0558841
:100AF00001D055988150CF0B8F0A20E1060E546E1D
:100B0000130E536EAE0EE82EFED7532EFCD7542E86
:100B1000FAD78150CF0B8F0AFCE055BE02D0558E1C
:100B200001D0559E060E546E130E536EAE0EE82E77
:100B3000FED7532EFCD7542EFAD7FF000EEC16F03A
:100B4000C06F39EC1CF099EC0BF00001B75108E0D4
:100B5000B751800A7F0F02E325DB02D0B7BF26DB47
:100B600098EC19F05C6E0001D651C0190CE1010E31
:100B700055AC000E536E010E55AE000E531A03E134
:100B8000BD515C1802E0B8EC1CF00EEC16F0C06F22
:100B90004ED0C00E846FF30E856F5E0E866F010E11
:100BA000876F806B3F0E816FAB0E826F010E836F7C
:100BB000040E21D03CDA28DA080E1DD038DA24DA07
:100BC0006C0E19D0846B856B866B1EDA700E13D099
:100BD000010E846F856B866B876BFE0E806F81695B
:100BE000826B836B0C0E07D029DAA3DA100E03D0C8
:100BF00025DA9FDA120EBF6F30D020DA030E7EDACC
:100C0000600E0ED01BDA030E79DA610E09D016DA07
:100C1000010E74DA620E04D011DA020E6FDA630E7E
:100C2000BF6F010E0BEC18F0700ED46F16D05C5035
:100C3000B0E0010ABFE0030AC1E0010AC3E0070A0D
:100C4000C7E0010AD1E0030AD3E0010AD6E00F0AA7
:100C5000D9E0010ADCE0030ADFE0040E5C600BD09F
:100C6000BF51E4EC18F006C056F007C057F008C0BA
:100C700058F009C059F0040E5C1806E0050E5C1827
:100C800003E0060E5C180AE10001BF511FEC1CF0E6
:100C900006C056F007C057F0586A596A060E5C64E1
:100CA00008D00001BF5119EC1DF0566E576A586A02
:100CB000596A0001D70509E1C4515626C55157228A
:100CC000C6515822C7515922D76BEDD908E280C0CE
:100CD00056F081C057F082C058F083C059F0020E20
:100CE000D71909E1C451565EC551575AC651585AD1
:100CF000C751595AD76B8451565C85515758865104
:100D000058588751595802E3CED908E284C056F0AA
:100D100085C057F086C058F087C059F0040ED71927
:100D20002EE0A05156182BE1A151571828E1A251ED
:100D3000581825E1A351591822E1010E55A8000EBB
:100D4000536E010E55A6000E531A19E1010E55AC53
:100D5000000E536E010E55AE000E531A10E1BD5138
:100D60005C180DE1010E55AA000E536E010E55A040
:100D7000000E531A04E1D651C01901E1A9D00EECBE
:100D800016F0C06F39EC1CF00001BD515C1802E098
:100D9000B8EC1CF099EC0BF0050E5C600DD056C061
:100DA00042F057C043F058C044F059C045F0E8EC59
:100DB00014F00EEC16F0C06F040E5C600CD056C040
:100DC00006F057C007F058C008F059C009F0BFC07E
:100DD0000AF0CBEC1BF0040E5C1806E0050E5C1864
:100DE00003E0060E5C1808E156C006F057C007F095
:100DF000BFC008F0E9EC1CF0060E5C6406D056C0DB
:100E000004F00001BF5194EC1CF05C5020E156C08E
:100E1000CCF057C0CDF058C0CEF059C0CFF006D0BE
:100E2000D1D80BD0BED809D0DED807D00001C3512D
:100E3000F7E0010AF7E0030AF7E08BD81A0E406EDC
:100E4000E7EC08F0A5D8220E406EE7EC08F05C0451
:100E500013E18CD87ED81A0E406EE7EC08F098D8D3
:100E6000220E406EE7EC08F056C094F057C095F0A3
:100E700058C096F059C097F0020E5C1813E176D86E
:100E800068D81A0E406EE7EC08F082D8220E406E49
:100E9000E7EC08F056C090F057C091F058C092F0BF
:100EA00059C093F0030E5C1813E160D852D81A0EA3
:100EB000406EE7EC08F06CD8220E406EE7EC08F0CC
:100EC00056C08CF057C08DF058C08EF059C08FF0CE
:100ED000040E5C182CE156C0ACF057C0ADF097EC96
:100EE00013F042D920EC13F030D9260E046E000E18
:100EF000F7EC1CF0D50E406E7F0E416E9BEC1AF0A5
:100F0000F5D841EC1BF0AFD809EC14F0FCD89BEC01
:100F10001AF0E4D8ACEC1BF0ADD809EC14F0A80E34
:100F2000406E7F0E416E9BEC1AF099EC0BF0040EB4
:100F30000001D71906E1C5EC17F00E6AD45198EC00
:100F400012F00001D76B010EC16F55AE07EF00F034
:100F5000C1D59C51C8253C6E9D51C9213D6E9E5105
:100F6000CA213E6E9F51CB213F6E120056C09CF0AD
:100F700057C09DF058C09EF059C09FF056C098F0E1
:100F800057C099F058C09AF059C09BF00001120068
:100F900098C03CF099C03DF09AC03EF09BC03FF035
:100FA000120090C09CF091C09DF092C09EF093C042
:100FB0009FF090C098F091C099F092C09AF093C0C1
:100FC0009BF0120094C09CF095C09DF096C09EF0DE
:100FD00097C09FF094C098F095C099F096C09AF091
:100FE00097C09BF012008CC09CF08DC09DF08EC00D
:100FF0009EF08FC09FF08CC098F08DC099F08EC08D
:101000009AF08FC09BF01200876B800E806FC30E2A
:10101000816FC90E826F010E836F010C260E2E6E3A
:10102000530E2F6E090E306E010E316E000CA00EA5
:10103000846F860E856F010E866F010C846B856B45
:10104000866B876B1200C8C006F0C9C007F0CAC023
:1010500008F0CBC009F0BFC00AF01200076E0A6AA0
:10106000800E096E800C04C040F005C041F0426A59
:10107000436A120004C040F005C041F0426A436A6E
:1010800012005CC0BDF0C3C0C2F055A002D0558AAA
:101090001200559A1200280E386EB0C039F0B1C057
:1010A0003AF03B6A020C5650805D575081595850B7
:1010B0008259595083591200C8C088F0C9C089F0BC
:1010C000CAC08AF0CBC08BF0120056C0A0F057C047
:1010D000A1F058C0A2F059C0A3F01200AEC004F0B5
:1010E000AFC005F0076A0A0E066E0A0CAEC004F027
:1010F000AFC005F0076A0A0E066E0A0C806F816B9E
:10110000826B836B12003D0E406E7F0E416E1200AB
:10111000F60E406E7F0E416E1200536E010E55A00A
:10112000000E531A1200536E010E55A0000E531AF2
:101130001200806BFA0E816F826B836BFA0C1A0EB1
:101140000001BC6F220EBB6F220C3CC0AEF03DC054
:10115000AFF01200096E0A6A000E0A22000CF90EA6
:10116000406E7F0E416E12003CC0AAF03DC0ABF055
:101170001200C00E386E7E0E396E1200076A0A0E1B
:10118000066E0A0C0F0E426E360C1A0E426E360CAC
:10119000076A060E066E060C1A0E426E000C0F0E43
:1011A000046E1E0C010ED76FB707010C020ED76F2D
:1011B000B72B020C030E046E000C0F0E426E000CD7
:1011C0001A0E046E1E0C076E0A6A096A12000101EB
:1011D000676B010E666F100E4024686F696B000E1E
:1011E0006923120E40244D6F4E6B000E4E23046A8D
:1011F000E90E056EA40E066E350E076E3CC008F0B3
:101200003DC009F03EC00AF03FC00BF023EC19F0DE
:1012100004C05FF105C060F106C061F107C062F172
:1012200008D0D89066376737D8906233613360331F
:101230005F33010162516111F4E1850E5F5D030EC0
:101240006059EFE25FA105D05F07000E605B615B54
:10125000625B66C104F067C105F0066A076A5FC198
:1012600008F060C109F061C10AF062C10BF0F5EC51
:101270001AF004C03CF105C03DF106C03EF107C0C4
:101280003FF13CC104F03DC105F03EC106F03FC155
:1012900007F03CC008F03DC009F03EC00AF03FC076
:1012A0000BF0F5EC1AF004C043F105C044F106C0A0
:1012B00045F107C046F121D00101666B676B34D060
:1012C0000101676B100E17D00101676B200E13D060
:1012D0000101676B300E0FD00101676B400E0BD020
:1012E0000101676B500E07D00101676B600E03D0E0
:1012F0000101676B700E666F17D066C141F067C160
:1013000042F0425011E14150010AD6E0030AD8E010
:10131000060ADAE00C0ADCE0180ADEE0300AE0E057
:10132000600AE2E0C00AE4E043C104F044C105F011
:1013300045C106F046C107F0CCC008F0CDC009F0A9
:10134000CEC00AF0CFC00BF023EC19F004C04BF173
:1013500005C04CF14BC104F04CC105F0066A076AA8
:10136000CCC008F0CDC009F0CEC00AF0CFC00BF061
:10137000F5EC1AF004500101435D116E055044591B
:10138000126E06504559136E07504659146E1BECE9
:101390001BF0C1D963C10FF064C110F065C111F039
:1013A000126A800E136E490E146E4CEC15F00FC0CD
:1013B00063F110C064F111C065F163C11EF064C136
:1013C0001FF065C120F0CCC011F0CDC012F0CEC02E
:1013D00013F0CFC014F01BEC1BF011C021F012C0B1
:1013E00022F013C023F0C7EC16F01EC063F11FC03B
:1013F00064F120C065F196D96BEC16F02DC047F171
:101400002EC048F12FC049F130C04AF15FC141F010
:1014100060C142F061C143F062C144F0070E75D96A
:10142000E82EFDD7000E41240101536FFE0E42202D
:10143000546FFF0E4320556FFF0E4420566FFE0E73
:10144000086E09680F0E0A6E0B6A4DD95ED9E82E38
:10145000FDD741C004F042C005F043C006F044C0CF
:1014600007F023EC19F004C011F005C012F006C01B
:1014700013F007C014F01BEC1BF04DD963C112F040
:1014800064C113F065C114F04BC141F04CC142F08E
:10149000070ED89041364236E82EFBD741C00CF0FB
:1014A00042C00DF0A6EC1CF00CC00FF00DC010F007
:1014B0000EC011F0C8EC10F00FC040F110C041F1A7
:1014C00011C042F1126A136AC40E146E40C10FF0CB
:1014D00041C110F042C111F0C8EC10F00FC02DF066
:1014E00010C02EF011C02FF06BEC16F02DC057F18C
:1014F0002EC058F12FC059F130C05AF113D96BECFE
:1015000016F02DC05BF12EC05CF12FC05DF130C034
:101510005EF15BC104F05CC105F05DC106F05EC127
:1015200007F0020E086E096AF00E0A6E0B68F5EC01
:101530001AF0D9D8EAD8E82EFDD704504124010189
:101540005B6F055042205C6F065043205D6F075073
:1015500044205E6FFE0E4F6F50690F0E516F526B3D
:1015600040C007F0086A5051096E0A6A6BEC1CF023
:101570004028076E086A000E082201014F51096ECB
:101580000A6A6BEC1CF0020EA8D8030E0101591573
:10159000096E0A6A6BEC1CF0030E9FD801015851CA
:1015A000096E0A6A6BEC1CF0040E97D801015751C2
:1015B000096E0A6A6BEC1CF0050E8FD80F0E010144
:1015C0005D15416E426A4FC143F050C144F051C1B4
:1015D00045F052C146F00D0E05D0D8904632453246
:1015E00044324332E82EF9D7F00E4316446A415094
:1015F0004310096E425044100A6E6BEC1CF0060E4C
:101600006CD801015C51096E0A6A6BEC1CF0070E84
:1016100064D801015B51096E0A6A6BEC1CF068C169
:1016200007F069C108F00A6A096A6BEC1CF0010E48
:101630004DD80A6A010E096E6BEC1CF0020E46D8FA
:10164000030E5515416E426A6611096E67514210CC
:101650000A6E6BEC1CF0030E39D85451096E0A6AFD
:101660006BEC1CF0040E32D85351096E0A6A6BEC15
:101670001CF0050E2BD80A6A096A6BEC1CF0060EEA
:1016800025D80A6A096A6BEC1CF0070E1FD80A6A93
:10169000096A6BEC1CF0040E01015F196011611105
:1016A0006211D8A412004DC107F04EC108F00C0E13
:1016B0006611096E67510A6E6BEC1CF0010E1CD8A6
:1016C0006BEC1CF0020E18D86BEF1CF001016825C2
:1016D000076E000E6921086E12004024076E086A2A
:1016E000000E0822000C47C141F048C142F049C138
:1016F00043F04AC144F0070C01014D25076E000E6E
:101700004E21086E0A6A096A1200D89041364236A4
:1017100043364436120011C063F112C064F113C0A5
:1017200065F1120063C12DF064C12EF065C12FF088
:10173000120039EC1CF0010E2BEC1DF0CAD9F7ECAD
:101740001CF064D1310E406E7F0E17D0C60E406E75
:101750007E0E13D0D60E406E7E0E0FD0F50E406E6C
:101760007E0E0BD0E60E406E7E0E07D0900E406EC1
:101770007F0E03D09C0E406E7F0E416E9BEF1AF0E1
:10178000000E046AF7EC1CF0040E406E7F0E416EF2
:101790009BEC1AF09BD9F7EC1CF06BD907E15CD9F4
:1017A00032EC1DF061D99BEC1AF007D0046A010EEF
:1017B00032EC1DF059D99BEC1AF0140E046EF7ECC4
:1017C0001CF061D907E148D932EC1DF048D99BECF7
:1017D0001AF007D0046A010E32EC1DF040D99BECE0
:1017E0001AF07DD9F7EC1CF0020E31D907E134D99B
:1017F00032EC1DF043D99BEC1AF007D0046A010EBD
:1018000032EC1DF03BD99BEC1AF066D9F7EC1CF0DA
:10181000030E1DD907E120D932EC1DF039D99BEC1C
:101820001AF007D0046A010E32EC1DF031D99BEC9E
:101830001AF0046A010E32EC1DF039EF1CF0000EB4
:10184000046AF7EC1CF0130E406E7F0E416E9BECA9
:101850001AF03CD9F7EC1CF00CD907E1FDD832ECBA
:101860001DF002D99BEC1AF007D0046A010E32EC8D
:101870001DF0FAD89BEC1AF0140E046EF7EC1CF075
:1018800002D907E1E9D832EC1DF0E9D89BEC1AF057
:1018900007D0046A010E32EC1DF0E1D89BEC1AF07F
:1018A0001ED9F7EC1CF0020ED2D807E1D5D832ECE5
:1018B0001DF0E4D89BEC1AF007D0046A010E32EC5C
:1018C0001DF0DCD89BEC1AF007D9F7EC1CF0030EE6
:1018D000BED807E1C1D832EC1DF0DAD89BEC1AF083
:1018E00007D0046A010E32EC1DF0D2D89BEC1AF03E
:1018F000046A010E32EC1DF039EF1CF0000E046A90
:10190000F7EC1CF04D0E406E7F0E416E9BEC1AF012
:10191000E0D8F7EC1CF0B7D807E19ED832EC1DF008
:10192000C1D89BEC1AF007D0046A010E32EC1DF00E
:10193000B9D89BEC1AF0240E046E000EF7EC1CF0E4
:1019400098D807E189D832EC1DF0B1D89BEC1AF099
:1019500007D0046A010E32EC1DF0A9D89BEC1AF0F6
:10196000046A010E32EC1DF039EF1CF0000E046A1F
:10197000F7EC1CF03F0E406E7F0E416E9BEC1AF0B0
:10198000140E046E000EF7EC1CF073D807E164D857
:1019900032EC1DF096D89BEC1AF007D0046A010EC9
:1019A00032EC1DF08ED89BEC1AF01E0E046E000E69
:1019B000F7EC1CF068D807E14FD832EC1DF07CD86A
:1019C0009BEC1AF007D0046A010E32EC1DF074D8BB
:1019D0009BEC1AF0280E046E000EF7EC1CF0020EC1
:1019E00036D807E139D832EC1DF057D89BEC1AF005
:1019F00007D0046A010E32EC1DF04FD89BEC1AF0B0
:101A0000046A010E32EC1DF039EF1CF05C5001E16C
:101A100099D6010A01E19AD6030A01E19BD6010A8F
:101A200001E19CD6070A01E19DD6010A01E19ED69B
:101A3000030A01E19FD6010A01E1A2D60F0A01E1E2
:101A4000FED6010A01E15AD7030A90E012005618A7
:101A50005710581059101200010E046E000CBD0EE4
:101A6000406E7F0E416E1200B70E406E7F0E416ECB
:101A7000120056505710581059101200C30E406EE5
:101A80007F0E416E12005604571058105910120064
:101A9000C90E406E7F0E416E12005B0E406E7F0ECF
:101AA000416E1200830E406E7F0E416E1200220EB8
:101AB000406E7F0E416E1200760E406E7F0E416EBC
:101AC0001200690E406E7F0E416E12000A0E046E07
:101AD000140C180E046E000C280E046E140C1E0E4E
:101AE000046E140C086AE80E096E760E0A6E480E33
:101AF0000B6E13D923EC19F002D96AEC1AF01150CD
:101B0000226E086AE40E096E0B0E0A6E540E0B6EFE
:101B100004D923EC19F0F3D86AEC1AF01150236EB3
:101B2000086ACA0E096E9A0E0A6E3B0E0B6EF5D845
:101B300023EC19F0E4D86AEC1AF01150246E086A0C
:101B4000E10E096EF50E0A6E050E0B6EE6D823EC5B
:101B500019F0D5D86AEC1AF01150256E800E086E77
:101B6000960E096E980E0A6E0B6AD7D823EC19F000
:101B7000C6D86AEC1AF01150266E400E086E420E5E
:101B8000096E0F0E0A6E0B6AC8D823EC19F0B7D88D
:101B90006AEC1AF01150276EA00E086E860E096EC0
:101BA000010E0A6E0B6AB9D823EC19F0A8D86AECBA
:101BB0001AF01150286E100E086E270EBCD8ADD842
:101BC00023EC19F09CD86AEC1AF01150296EE80E3B
:101BD000086E030EB0D8A1D823EC19F090D86AECA7
:101BE0001AF011502A6E640EA1D897D823EC19F080
:101BF00086D86AEC1AF011502B6E0A0E97D88DD841
:101C000023EC19F07CD86AEC1AF011502C6E1AC033
:101C100011F01BC012F01CC013F01DC014F00A0E0E
:101C2000156E166A176A186A6AEC1AF011502D6E52
:101C3000306A316A3050220FD96EDA6A3050220F82
:101C4000E16EE26AE750300FDF6E304A312A31BE72
:101C5000F1D7315003E10C0E305CECE3306A316AAD
:101C600002D0304A312A79D8300EDE1807E131BE71
:101C7000F8D7315003E1050E305CF3E320500C0837
:101C80002E6E000ED8A0E82A00082F6E10D060D863
:101C9000200EDF6E080E2E182F1004E0050E2E18F1
:101CA0002F1001E14CD81E4A1F2A2E4A2F2A3050ED
:101CB0002E5C2F50800A216E3150800A2158E7E3B4
:101CC00031BE05D0315018E10C0E305C15E245D81C
:101CD0001EC0E1FF1FC0E2FFDFCFE7FF080E301894
:101CE000311004E0050E3018311001E128D81E4AE9
:101CF0001F2A304A312AE4D72BD8DF6A000C04C0EF
:101D000011F005C012F006C013F007C014F00A0E5F
:101D1000156E166A176A186A0A0C1AC004F01BC0FE
:101D200005F01CC006F01DC007F01200086E096A1D
:101D30000A6A0B6A1200096E0A6A0B6A12001E4ACE
:101D40001F2A1EC0D9FF1FC0DAFF2E0EDF6E2E0C19
:101D50001EC0D9FF1FC0DAFF12003050220FD96E0B
:101D6000DA6A12003F6E070E3F1804E10001B56BFE
:101D70005B6A1200200E3F1803E15B5001E1120084
:101D8000080E3F1813E15A50060D5B50386E396A41
:101D9000F350385C3950800A3A6EF450800A3A5851
:101DA00005E35A50060DF3505B5E12000D0E3F180E
:101DB00002E15B6A12000A0E3F1811E1C2D85A50C4
:101DC000070DB551F326000EF422F4BE000CF450BA
:101DD00004E1310EF35CD8A01200B56B12001F0EA7
:101DE0003F6403D07E0E3F6402D03F0E3F6E3E6ADA
:101DF000600E386E39683F50050DE50E3A6E7C0E68
:101E00003B6EF3503A26F4503B223E503A26000EE9
:101E10003B2238503A2639503B223AC0F6FF3BC0AD
:101E2000F7FF0800F5CF3CF03D6A3CA013D05A0400
:101E300008E10001B5513D24A7D83E247AEC14F006
:101E40001FD03D5065D85DD8D2C031F093D88BEC0F
:101E50001BF016D00001D251B31912E05A0407E169
:101E6000B5513D248CD83E247AEC14F009D03D5075
:101E70005A02F35046D8B3C031F07CD88BEC1BF03B
:101E80003D2AD8903C32070E3D64CFD73E2A040E3F
:101E90003E64AED70001D251B31909E05A0404E1FF
:101EA00047D804EC1CF003D01DD88BEC1BF05CD899
:101EB000386E396A4CD830D802E2540E5B6E4DD879
:101EC000F4BE000CF45004E1550EF35CD8A01200EF
:101ED0005B6A37D8B551386E396A3CD81DD8D8B04E
:101EE000120057D0B5C02EF05AC02FF05A50080D2E
:101EF000F3CF30F0B3C031F05A50050DF3505B24EE
:101F00001200B5252E6E5AC02FF05AC030F01200C4
:101F10005A02F35000011200F326000EF42238504A
:101F2000F35CF450800A3A6E3950800A3A58120035
:101F3000B5C028F0080E296EB3C02AF05B50050F1B
:101F400012005A50080DF3500001B52712005A50E4
:101F5000060D540C5A50080D300C5A50050D5B50AC
:101F6000F326000EF422000C5A50060DF3505B26A7
:101F70005B5012003E505A02F3505B241200046E74
:101F8000B3C005F05B501200046ED2C005F05B5088
:101F90001200300EB56F300C000000000000000091
:101FA0000000000000000000000000000000000031
:101FB0000000000000000000000000000000C0E081
:101FC000F0F8FCFCFEFFFCE0000000000000000058
:101FD0000000000000000000000000000000000001
:101FE00000000000000000000000000000000000F1
:101FF00000000000000000000000000000F8F8F8F9
:10200000F8F8F8F8F8F8F8F8F8F0F0E0E0C080C078
:10201000FCFFFFFFFF7F3F7FFFFFFFFFFF00000090
:1020200000000000000000000000000000000000B0
:1020300000000000000000000000000000000000A0
:102040000000000000000000000000000000000090
:1020500000000F1F3F7FFFFFFFFFFFFFFFFFE7C7EE
:10206000C7878F9F9FFFFFFFC1C0E0FCFFFFFFFFFF
:10207000FFFCFCFCFCFEFEFEFCFCF8F8F0E0C0C03F
:102080000000000000000000000000000000000050
:102090000000000000000000000000000000000040
:1020A00000000000000000000080C0E0F1FBFFFF26
:1020B000FFFFFF7F1F0F0F87E7FFFFFF1F1F3FF986
:1020C000F8F8F8F8F8F8FDFFFFFFFFFFFFFFFFFF4C
:1020D0007F3F0F070100000000000000000000002B
:1020E00000000000000000000000000000000000F0
:1020F0000000000000000000000000F0FEFFFFFFF5
:10210000FFFFFFFFFFFFFFFE7E3F3F0F1FFFFFFFB1
:10211000FCF0E0F1FFFFFFFFFFFCF0010101010116
:1021200001010100000000000000000000000000AC
:10213000000000000000000000000000000000009F
:10214000000000000000000000000000000000038C
:102150000303030303030301010101000000000066
:102160000000030F1F3F7F7FFFFFFFFF7F7F1F03E5
:10217000000000000000000000000000000000005F
:10218000000000000000000000000000000000004F
:1021900011C015F0166A176A1034153601E316805F
:1021A00015501A6E14C015F0166A176A13341536D6
:1021B00001E316801550196E1A5009E019501A5C87
:1021C0000DE21A50195C156E180E156407D012C076
:1021D0000FF013C010F014C011F01200195009E0F4
:1021E0001A50195C0DE219501A5C156E180E156420
:1021F00007D00FC00FF010C010F011C011F0120086
:10220000060E186E11BE188E14BE188C108E116A30
:10221000138E146A19501A5C14E2D89012361336D1
:10222000143619061A50191808E053D806E0F5D7E5
:10223000D890113210320F321A2A19501A1817E09A
:10224000F7D71A50195C13E2D8900F3610361136B2
:102250001A061A50191808E03CD806E0F5D7D890AD
:10226000143213321232192A19501A18F8E118AE22
:1022700007D00F1E101E111E0F2A000E1022112251
:1022800018BC1FD8186A0F50122610501322115074
:10229000142214AE03D015D8010E186E12C004F02B
:1022A00013C005F014C006F01AC007F018C008F0FB
:1022B000A1EC18F004C00FF005C010F006C011F03A
:1022C0001200121E131E141E122A000E13221422B4
:1022D000000C180618C015F0070E1516070C0E5046
:1022E000125C046E0F501358056E80EC1CF004C095
:1022F00017F005C018F08BD880EC1CF00450175C68
:102300001850800A196E0550800A1958010ED8B06D
:10231000000E266E265018E00EC01AF00FC01BF0FB
:1023200010C00EF011C00FF01AC010F01BC011F059
:1023300012C01CF013C01DF014C012F015C013F031
:102340001CC014F01DC015F059D818E20EC01EF0C4
:102350000FC01FF012C00EF013C00FF01EC012F01D
:102360001FC013F010C020F011C021F014C010F0F5
:1023700015C011F020C014F021C015F00E50125CF1
:10238000276E45D880EC1CF00450226ED890273080
:10239000236E246A1450105C1150800A176E155079
:1023A000800A175803E2010E256E25D0256823D038
:1023B000265008E00EC004F016C005F010507AEC6C
:1023C00014F007D010C004F016C005F00E507AECDF
:1023D00014F02250235E000E245A24AE0AD0255059
:1023E0001026000E25BEFF0E112227502326000EB8
:1023F00024220E4A0F2A02D8DBE212000E50125C91
:102400001350800A176E0F50800A17581200105090
:10241000145C046E11501558056E12003F6A3F504F
:1024200038243A6E000E39203B6E3AC0F6FF3BC0AE
:10243000F7FF0800F5CF3DF03E6A3DA016D05A04E4
:1024400009E10001B5513E24C4EC0FF03F247AECC1
:1024500014F023D03E5088EC0FF081EC0FF0D2C086
:1024600031F061D88BEC1BF018D00001D251B319B8
:1024700014E05A0408E1B5513E24BFEC0FF03F24AC
:102480007AEC14F00AD03E505A02F35081EC0FF06F
:10249000B3C031F048D88BEC1BF03E2AD8903D32C7
:1024A000070E3E64CAD73F2A040E3F64B8D7000126
:1024B000D251B3190BE05A0405E198EC0FF004EC8B
:1024C0001CF004D072EC0FF08BEC1BF0B4EC0FF0AE
:1024D0003A6E3B6AA7EC0FF01AD802E2540E5B6E1C
:1024E000ADEC0FF0F4BE000CF45004E1550EF35CBB
:1024F000D8A012005B6AA1EC0FF0B5513A6E3B6AAE
:10250000AAEC0FF004D8D8B01200C9EF0FF0F326F0
:10251000000EF4223A50F35CF450800A3C6E3B50BB
:10252000800A3C5812003F505A02F3505B241200BC
:10253000156E55AE05D0060E5C6402D05596060C9D
:10254000136A146A0E5005E1186A196A126A020EBB
:1025500004D0196A010E186E126A116E166A176A93
:1025600039D01A6A1B6A05D066D87AEC14F01A4A78
:102570001B2A155018240F6E000E1920106E56D805
:10258000F3E3155018241A6E000E19201B6E09D0A3
:1025900016C004F0010E056E1A507AEC14F01A4AB7
:1025A0001B2A3CD80F26000E102240D8F1E336D863
:1025B0000F241A6E000E10201B6E05D03CD87AEC4A
:1025C00014F01A4A1B2A1B5003E1540E1A5CF6E35E
:1025D000164A172A115013240F6E12501420106E31
:1025E0000F50165C10501758BCE30E5002E139EF43
:1025F0001CF01A6A1B6A09D013501124046E056A74
:102600001A507AEC14F01A4A1B2A1B5002E039EFD8
:102610001CF0540E1A5CF0E339EF1CF015500F6EED
:10262000106A18500F5E1950105A050C0F501A5CA2
:1026300010501B58120016C004F0056A1A50120000
:10264000010E38EC1AF00BC044F00CC045F0126AD1
:10265000480E136E420E146E44280C6E000E452078
:102660000D6EA6EC1CF04ED84CEC15F052D8216A39
:10267000800E226E440E236EC7EC16F01EC046F08C
:102680001FC047F020C048F04BD8ACC00CF0ADC024
:102690000DF0A6EC1CF036D84CEC15F00FC03EF057
:1026A00010C03FF011C040F03BD83EC00FF03FC01B
:1026B00010F040C011F04CEC15F00FC041F010C00C
:1026C00042F011C043F0F40E216EA10E226E470EAF
:1026D000236E126A800E136E3F0E146E41C00FF00F
:1026E00042C010F043C011F04CEC15F012D8C7EC0A
:1026F00016F0F8EC13F06BEC16F02DC03CF02EC089
:102700003DF012000CC00FF00DC010F00EC011F023
:1027100012000FC01EF010C01FF011C020F01200F8
:1027200046C012F047C013F048C014F01200010E6A
:1027300038EC1AF00BC03EF00CC03FF0020E38EC43
:102740001AF00BC040F00CC041F059D817E34050CC
:102750003E5C0C6E41503F580D6EA6EC1CF036D816
:10276000A6EC1CF082EC13F04CEC15F089EC13F0A5
:10277000C7EC16F03DD86BEC16F046D840D817E2FF
:102780003E50405C0C6E3F5041580D6EA6EC1CF064
:102790001DD8A6EC1CF082EC13F04CEC15F089EC83
:1027A00013F0C7EC16F024D86BEC16F02DD8E80E19
:1027B0000001AA5D030EAB5904E3030EAB6FE70EF5
:1027C000AA6FAAC03CF0ABC03DF012000CC021F0D3
:1027D0000DC022F00EC023F0126A200E136E410EBF
:1027E000146E40503E240C6E41503F200D6E12007E
:1027F0001EC02DF01FC02EF020C02FF01200405040
:102800003E5C41503F5812002DC0AAF02EC0ABF0E4
:102810001200526A405041104210431003E1300E42
:10282000B2EF0EF043AE39D02D0EB2EC0EF0431ED7
:10283000421E411E406C000E4122422243222DD0F6
:102840005250460FD96EDA6A40C004F041C005F01C
:1028500042C006F043C007F00A0E086E096A0A6A11
:102860000B6A78EC17F00450DF6E522A40C004F077
:1028700041C005F042C006F043C007F00A0E086EE2
:10288000096A0A6A0B6AB0EC15F004C040F005C092
:1028900041F006C042F007C043F043BE09D04350A8
:1028A0004210411002E1400403E30A0E5264C8D70B
:1028B000525001E1120016D8090EDF6405D012D87B
:1028C000DF50456E370E04D00DD8DF50456E300E08
:1028D0004524506E516A000E51225050B2EC0EF059
:1028E0005206E6D752C044F044064450460FD96E13
:1028F000DA6A12000D6E540E0D60540C2F0E046433
:1029000018D02F0C0DC00BF00C6A04C00DF00B504A
:1029100004D00D5053080D6E04502F08046E11D0D2
:102920000DC00BF00C6A045053080D6E0BC004F080
:1029300008D00001B451010AE5E0030AEAE0010A07
:10294000EFE0540E0D60540C2F0E046401D02F0CD8
:10295000055017E02FD802D0D8900736062EFCD7A6
:1029600031D8086E010E096EF3500826F450092282
:102970000D500824D96E000E0920DA6E0750DF12C0
:10298000120018D802D0D8900736062EFCD7071CA4
:10299000086E18D8096E010E0A6EF3500926F4501D
:1029A0000A220D500924D96E000E0A20DA6E085052
:1029B000DF16120004C006F0070E0616010E076EA1
:1029C000062A010C0438E8461F0B540D6A0E12004B
:1029D000455007E1800E425C960E4358980E4458CD
:1029E00016E3DAEC08F0F7EC1CF02CD872EC0DF0E2
:1029F00044D89BEC1AF055BE05D03AD89BEC1AF09F
:102A000039EF1CF03FD89BEC1AF039EF1CF0030EA5
:102A100028D88BEC1BF0030E046E060EF7EC1CF0AE
:102A200011D872EC0DF033D89BEC1AF055BE05D0DE
:102A30001FD89BEC1AF039EF1CF024D89BEC1AF04D
:102A400039EF1CF042C01AF043C01BF044C01CF028
:102A500045C01DF0000E1E6E010E1F6E080E206E8A
:102A6000080C2E6E060E2F6E080E306E316A000CAA
:102A7000DF0E406E7F0E416E1200000E406E010EA2
:102A8000416E1200DA0E406E7F0E416E1200010E92
:102A9000406E010E416E120011C015F0166A176AE1
:102AA0001034153601E316801550186E185001E1E8
:102AB00053D014C015F0166A176A1334153601E3A3
:102AC000168015501D6E1D5001E146D01D507B0F24
:102AD000182611C01DF014501D1A800E1D16108EE0
:102AE000138E000E1416196A1A6A1B6A070E1C6EE2
:102AF0000FB02BD8D890113210320F32D890123636
:102B0000133614361C2EF4D7090E1C6E0FB01DD8C8
:102B1000D890113210320F32D8901B321A3219323B
:102B20001C2EF4D719C004F01AC005F01BC006F023
:102B300018C007F01DC008F0A1EC18F004C00FF099
:102B400005C010F006C011F01200125019261350E3
:102B50001A2214501B2212000F6A106A116A120006
:102B60000D6A0BAE0AD00B1E0A1E091E086C000E61
:102B700009220A220B22010E0D6E07AE0AD0071E93
:102B8000061E051E046C000E052206220722010EF9
:102B90000D1A0E6A0F6A106A116A085009100A109D
:102BA0000B1029E0010E0C6E06D0D89008360936BD
:102BB0000A360B360C2A0BAEF8D7D8900E360F36E5
:102BC000103611360850045C095005580A50065852
:102BD0000B50075809E30850045E0950055A0A5083
:102BE000065A0B50075A0E80D8900B320A3209321F
:102BF00008320C2EE2D70D5008E0111E101E0F1ED9
:102C00000E6C000E0F22102211220EC004F00FC015
:102C100005F010C006F011C007F0120055AE02D04A
:102C2000070E1E6E55BE02D0050E1E6EC0C0D6F039
:102C30008150CF0BCE0A15E10001C0071E50C05DC8
:102C400001E3C06B060E1D6E130E1C6EAE0EE82E59
:102C5000FED71C2EFCD71D2EFAD78150CF0BCE0AE3
:102C6000FCE08150CF0BCC0A16E10001C02B1E50B6
:102C7000C05D02E31EC0C0F0060E1D6E130E1C6E7A
:102C8000AE0EE82EFED71C2EFCD71D2EFAD7815093
:102C9000CF0BCC0AFCE0C5EC17F00E6AD45198ECCF
:102CA00012F00001D651C01913E055BE11D0C0C0BA
:102CB00004F0000E94EC1CF0030E1D6E080E1C6E4A
:102CC000770EE82EFED71C2EFCD71D2EFAD700F06B
:102CD0000001C05112002FC031F0326A336A2E3425
:102CE000313601E3328031503B6E3B5005E12D6AB5
:102CF0002E6A2F6A306A1200170E316E2DC032F024
:102D00002EC033F02FC034F03128356E04D0D89067
:102D1000343233323232352EFAD73250366E2E8E6E
:102D20002F6A2D50376E2E50386E2F50396E3A6AFA
:102D30008E0E3B5E3BAE0CD03B50800A8F0FD7E32C
:102D4000D8903A323932383237323B3EF9D70CD04C
:102D5000170E3B6407D0CBD7D89037363836393684
:102D60003A363B063B50F8E1365008E03A1E391E31
:102D7000381E376C000E382239223A2237C02DF027
:102D800038C02EF039C02FF03AC030F0120020C009
:102D900024F0256A266A1F34243601E32580245056
:102DA0002B6E2B5001E14AD023C024F0256A266AFD
:102DB0002234243601E3258024502C6E2C5001E16E
:102DC0003DD0286A296A2A6A2C50890F2B5E20C0C0
:102DD0002CF023502C1A800E2C161F8E206A228E67
:102DE000236A180E276ED890283629362A362150A5
:102DF0001E5C22501F582350205807E321501E5EAE
:102E000022501F5A2350205A2880D8901E361F3631
:102E10002036272EE8D728C004F029C005F02AC0A4
:102E200006F02BC007F02CC008F0A1EC18F004C08D
:102E30001EF005C01FF006C020F012001E6A1F6AB7
:102E4000206A120055B004D00001BF51040F03D016
:102E50000001BF51FC0F426E4250E4EC18F006C076
:102E600043F007C044F008C045F009C046F04650A2
:102E700007E1800E435C960E4458980E455812E3C5
:102E80000F0E046E000EF7EC1CF023D872EC0DF060
:102E90003DEC15F09BEC1AF038EC15F09BEC1AF0B9
:102EA00039EF1CF00F0E31EC15F08BEC1BF00F0E10
:102EB000046E060EF7EC1CF00CD872EC0DF047EC2B
:102EC00015F09BEC1AF038EC15F09BEC1AF039EF8A
:102ED0001CF043C01AF044C01BF045C01CF046C0B3
:102EE0001DF0000E1E6E010E1F6E080E206E080CE7
:102EF0000D6A07AE03D040D8010E0D6E0BAE08D0A0
:102F00000B1E0A1E091E086C000E09220A220B2243
:102F1000085009100A100B1023E0010E0C6E06D0A9
:102F2000D890083609360A360B360C2A0BAEF8D77D
:102F30000850045C095005580A5006580B500758B1
:102F400008E30850045E0950055A0A50065A0B500F
:102F5000075AD8900B320A32093208320C2EE8D7C1
:102F60000D5001E009D804C004F005C005F006C00A
:102F700006F007C007F01200071E061E051E046CAF
:102F8000000E052206220722000C35D0010E43D880
:102F9000360ED46F360C0A0E3ED8300ED46F300C7D
:102FA000640E39D82A0ED46F2A0CE80EC46F030EB3
:102FB000C56FC66BC76B1E0ED46F1E0C100EC46F90
:102FC000270EC56FC66BC76B180ED46F180CA00EFA
:102FD000C46F860EC56F010EC66FC76B120ED46F1D
:102FE000120C400EC46F420EC56F0F0EC66FC76B3A
:102FF000060ED46F060C0001C051C8E0010ACBE0F8
:10300000030ACEE0010AD1E0070AD8E0010ADFE0B6
:10301000030AE7E01200C46FC56BC66BC76B1200F2
:103020003F6E3F503924406E000E3A20416E4150B1
:1030300003E1510E405C04E3000E416E500E406E01
:103040003B501BE127D88BEC1BF03FC03EF00AD071
:1030500038C02EF0030E2F6E27D83E508BEC1BF09D
:10306000050E3E263E503C6E3D6A40503C5C415051
:103070003D5802E339EF1CF0EBD70CD88BEC1BF07A
:1030800038C02EF040C02FF00FD83F288BEC1BF03B
:1030900039EF1CF038C02EF0405050082F6E050E4E
:1030A000306E316A40281200050E306E010E316E0E
:1030B000010C980EF66E1F0EF76E000EF86E01EE04
:1030C0006AF011EEF8F00900F5CFEEFFE550E1509F
:1030D000FAE1E250F8E11E0EF66E3A0EF76E000EBF
:1030E000F86E00EEC4F010EE14F00900F5CFEEFF1C
:1030F000E550E150FAE1940EF66E3A0EF76E000ECE
:10310000F86E00EE56F010EE05F00900F5CFEEFF78
:10311000E550E150FAE101EE00F03C0EEE6AE806FF
:10312000FDE100EE80F0440EEE6AE806FDE1556A2E
:103130005C6A5B6A5D905D92000EF86E000109EFBB
:1031400000F0075004E004500510061006E1046A80
:10315000056A066A1200072A32D8096A0A6AFE0E50
:10316000061428D807E0F7D7072A042A000E0522FC
:10317000062225D8096A0A6A06501CD806E0F4D748
:103180000706D89004360536063605BE03D0020E73
:103190000760F6D707A0059ED890073207500612A1
:1031A000085001E0068E04C004F005C005F006C01A
:1031B00006F012000B6E09500A100B101200D89086
:1031C0000632053204321200126E125019EC1DF054
:1031D0000E6E122819EC1DF00F6E1250020F19EC32
:1031E0001DF0106E1250030F19EC1DF0116E136AD2
:1031F000146A156A166A0E501326000E1422152240
:1032000016220F500DD810500BD8115009D813C0EA
:1032100006F014C007F015C008F016C009F012003F
:1032200013C00BF014C00CF015C00DF00A6A0A248C
:10323000136E000E0B20146E000E0C20156E000E87
:103240000D20166E12000C6A0D6A0E6A0F6A085085
:1032500009100A100B1029E0010E106E06D0D8904C
:10326000083609360A360B36102A0BAEF8D7D89036
:103270000C360D360E360F360850045C09500558D2
:103280000A5006580B50075809E30850045E0950CD
:10329000055A0A50065A0B50075A0C80D8900B3228
:1032A0000A3209320832102EE2D70CC004F00DC0E9
:1032B00005F00EC006F00FC007F012000600F2A0E5
:1032C00021D081AA03D0016A012A01D0016A81A814
:1032D00003D0026A022A01D0026AD8900234011097
:1032E000036E0001B25109E1030402E1010E04D0B2
:1032F000020E031802E1020ED76F03C0B2F081CFB5
:1033000081FFF2909EA012D00001D007D8A0D10773
:10331000D051D11108E1D16B960ED06F55B402D0C7
:10332000558401D055949E90CE6ACF6A5D9211006B
:1033300055BE02D0020E03D055AE02D00B0E3A6E2F
:103340008150CF0BC70A26E15C2A3A505C5C01E34E
:103350005C6A060E396E130E386EAE0EE82EFED77E
:10336000382EFCD7392EFAD78150CF0BC70AFCE094
:10337000030E2E6E520E2F6E0B0E0ED88BEC1BF022
:103380000F0E2E6E520E2F6E080E06D88BEC1BF011
:1033900039EC1CF05C501200306E316A000C086A87
:1033A000096A1A0E076EF80EE82EFED7072EFCD714
:1033B00000D0084A092A095003E1640E085CF1E3D1
:1033C00096928D920A6A0B6A1A0E076EF80EE82E14
:1033D000FED7072EFCD700D00A4A0B2A0B5003E178
:1033E000640E0A5CF1E38D82969092969298210E7B
:1033F0003DEC1DF0130E3DEC1DF0B20E3DEC1DF04A
:10340000200E3DEC1DF00C0E3DEF1DF0436E010E45
:103410002BEC1DF021D028D8F7EC1CF0E80E406E04
:103420007F0E416E9BEC1AF039EF1CF01DD8F7ECC3
:103430001CF0EC0E406E7F0E416E9BEC1AF039EFE3
:103440001CF012D8F7EC1CF0E40E406E7F0E416EBB
:103450009BEC1AF039EF1CF00001C351DCE0010ACB
:10346000E5E0030AEEE0120042C004F0435012000F
:10347000146E0F6A106A136A145002E1010EC26ED4
:10348000140402E1050EC26E020E141802E1090EC8
:10349000C26EC282C2B2FED7C4500E6E0D6AC35055
:1034A0000D24116E000E0E20126E11500F261250B8
:1034B0001022132A090E1364DFD70FC004F010C0C6
:1034C00005F0BEEC08F041EC1BF004C00BF005C0A9
:1034D0000CF01200155016101710181023E0010EF2
:1034E000196E06D0D8901536163617361836192AA2
:1034F00018AEF8D71550115C1650125817501358C3
:103500001850145808E31550115E1650125A1750EF
:10351000135A1850145AD8901832173216321532DE
:10352000192EE8D711C011F012C012F013C013F019
:1035300014C014F0120018D021D8F76403D008008A
:10354000F55001D022D8200A05E15B5003E1404A42
:10355000412A0AD013D8F76403D00800F55001D0EF
:1035600014D8B2EC0EF0F3D709D8F76403D00800F2
:10357000F55001D00AD80009DFE1120040C0F6FF83
:1035800041C0F7FFF86A050E1200F6CFE1FFF7CF52
:10359000E2FFE7501200280EC66EC56A046AB40E38
:1035A000056EC40E066E040E076E11C015F012C033
:1035B00016F013C017F014C018F0020ED89015368C
:1035C000163617361836E82EF9D715C008F016C08B
:1035D00009F017C00AF018C00BF023EC19F004042E
:1035E000C86EC76A9486948812000C6A0D6A0E6AC7
:1035F0000F6A04A008D008500C2609500D220A506A
:103600000E220B500F22D890083609360A360B3698
:10361000D8900732063205320432045005100610E5
:103620000710E7E10CC004F00DC005F00EC006F075
:103630000FC007F012008E0E196E06D0D89014320B
:10364000133212321132192A156A166A176A145087
:10365000186E1550161017101810F0E111C004F074
:1036600012C005F013C006F019C007F0000E086E76
:10367000A1EC18F004C011F005C012F006C013F060
:103680001200086A096A065007101BE0010E0A6E54
:1036900004D0D890063607360A2A07AEFAD7D89053
:1036A000083609360650045C0750055805E30650F5
:1036B000045E0750055A0880D890073206320A2E59
:1036C000EED708C004F009C005F01200336E2EC01A
:1036D00028F01BD8E9EC1BF02E503024326E320457
:1036E000286E13D8E9EC1BF008D804EC1CF005D8C0
:1036F0002F24326E320404EF1CF02EC028F030C0AC
:1037000029F031C02AF0335012002FC029F031C007
:103710002AF033501200356E35C036F0376A0BD0C0
:103720002EC028F030C029F031C02AF0365004EC09
:103730001CF0364A372A2F5035C032F0336A322611
:10374000000E33223250365C3750800A346E3350CC
:10375000800A3458E5E312000650071017E0010E06
:10376000086E04D0D89006360736082A07AEFAD776
:103770000650045C0750055804E30650045E0750E9
:10378000055AD89007320632082EF2D704C004F04A
:1037900005C005F0120009C00BF00BC004F00A5080
:1037A00094EC1CF008C00CF00CC004F00A2894EC57
:1037B0001CF007C00DF00DC004F00A50020F94EC8D
:1037C0001CF006C00EF00EC004F00A50030F94EF78
:1037D0001CF02D6E2DC00EF00F6A28C010F0116A7B
:1037E00029502DC02BF02C6A2B26000E2C22FF0E08
:1037F0002B24126EFF0E2C20136E28C014F0156AB5
:103800002AC016F06FEF11F02D6E2DC00EF00F6A6A
:1038100028C010F0116A2DC012F0136A295028C078
:103820002BF02C6A2B26000E2C22FF0E2B24146E5C
:10383000FF0E2C20156E2AC016F06FEF11F00A6EE5
:103840000A5019EC1DF00B6E0C6A0D6A0B500C2619
:10385000000E0D220A2819EC1DF00B6E0C50086E9C
:103860000B500C6E08C00DF00CC006F00DC007F038
:103870001200400E3DEC1DF0800E3DEC1DF08480EA
:10388000076A086A6A0E0724D96E010E0820DA6EEC
:10389000DF50C9EC1CF0074A082AF80E075C010E3D
:1038A0000858F0E31200436E42C004F04350F7ECB6
:1038B0001CF055B008D0B10E406E7F0E416E9BECEF
:1038C0001AF039EF1CF0CF0E406E7F0E416E9BEC6C
:1038D0001AF039EF1CF046EC1DF0066AC00E056EBA
:1038E00038EC1DF007C005F008C006F038EC1DF0FC
:1038F00009C005F00AC006F038EC1DF042EF1DF0DB
:1039000005AE0DD004C006F005C007F0061E071E68
:10391000064A072A06C004F007C005F0120004C0DA
:1039200004F005C005F01200056E05C0A9FF04C033
:10393000A8FFA69EA69CA684550EA76EAA0EA76EEB
:10394000A682A6B2FED7A198A69412000CC004F0DD
:103950000DC005F0066A8E0E076E000E086EA1EC13
:1039600018F004C00CF005C00DF006C00EF01200F7
:10397000046A056A6A0E0424D96E010E0520DA6E07
:10398000DF6A044A052AF80E045C010E0558F2E3CA
:103990001200046E800E056E0AD080980450051443
:1039A00002E0808601D080968088D890053205504C
:1039B000F4E11200076E7F0E076401D0076E210E3E
:1039C0003DEC1DF0075080093DEC1DF0200E3DEF51
:1039D0001DF007C009F009C004F0085094EC1CF079
:1039E00006C00AF00AC004F0082894EF1CF0056E27
:1039F000540E0560540C2F0E046401D02F0C05C02A
:103A00005BF004C0B5F012000F0E2E6E540E2F6E38
:103A1000210ECCEC19F08BEC1BF039EF1CF00100FF
:103A2000000060566C0040787D01500001528922F0
:103A30000704046E04C0A9FFA69EA69CA680A8CF7A
:103A400005F005501200C7B4FED7C5CF04F01F0E15
:103A50000416F9E11F0C046E045001E1120004C0C9
:103A60005AF01200056E05C0D2F004C0B3F0120087
:103A700023EC1DF005C0C9FF1200066E84900650AD
:103A8000C9EF1CF023EC1DF0C584120023EC1DF0DF
:103A9000C58012008096980001FFFFFFFFFFFFFF27
:103AA000FFFFFFFFFFFFFFFFFFFFFFFFFFFFFFFF26
:103AB000FFFFFFFFFFFFFFFFFFFFFFFFFFFFFFFF16
:103AC000FFFFFFFFFFFFFFFFFFFFFFFFFFFFFFFF06
:103AD000FFFFFFFFFFFFFFFFFFFFFFFFFFFFFFFFF6
:107CE000FFFFFFFF00000000000000005F00000039
:107CF00007000700147F147F147E7949797E3E04C3
:107D000004060636495620500008070300001C22CE
:107D100041000041221C002A1C7F1C2A08083E0842
:107D20000800807030000808080808000060600043
:107D300020100804023E5149453E00427F40007237
:107D4000494949462141494D331814127F102745AE
:107D50004545393C4A4949314121110907364949CC
:107D60004936464949291E000014000000403400ED
:107D700000000814224114141414140041221408A1
:107D800002015909063E415D594E7C1211127C7F59
:107D9000494949363E414141227F4141413E7F4967
:107DA0004949417F090909013E414151737F080852
:107DB000087F00417F41002040413F017F0814229D
:107DC000417F404040407F021C027F7F0408107FBB
:107DD0003E4141413E7F090909063E4151215E7FF6
:107DE00009192946264949493203017F01033F40C9
:107DF00040403F1F2040201F3F4038403F63140851
:107E0000146303047804036159494D43007F4141E1
:107E1000410204081020004141417F040201020494
:107E20004040404040000307080020545478407F01
:107E3000284444383844444428384444287F38543B
:107E400054541800087E090218A4A49C787F0804E2
:107E5000047800447D40002040403D007F102844CD
:107E60000000417F40007C047804787C080404789A
:107E70003844444438FC1824241818242418FC7C62
:107E800008040408485454542404043F44243C4047
:107E900040207C1C2040201C3C4030403C442810AA
:107EA00028444C9090907C4464544C4400083641E3
:107EB00000000077000000413608000201020402C1
:107EC0003844444438004C5342204652452E204FFB
:107ED000465345543A00555342204652452E204FB2
:107EE000465345543A00524620504F574552204B76
:107EF000414C2E3A004357204652452E204F4653C0
:107F000045543A00434C4B3020534556695945532C
:107F1000693A00434C4B31205345566959455369E2
:107F20003A0042656361796973206B6170616C69C5
:107F3000004B52695354414C204652454B2E004B46
:107F400052695354414C2E204B41502E0054782DF1
:107F500052782042454341596953004361702E20B5
:107F60003D3E203130207066004361702E203D3E42
:107F70002036207066004361702E203D3E20382060
:107F800070660042656361796973206163696B00A3
:107F90004F505369594F4E454C2031004F50536953
:107FA000594F4E454C2032002057617474202020D8
:107FB0000056464F2041003D3E326D41003D3E346B
:107FC0006D41003D3E366D41003D3E386D410056ED
:107FD000464F2042004755433A002020487A00206F
:107FE0004D487A00435720004C53420055534200FD
:0F7FF000503A00533A00525800545800240000F1
:020000040030CA
:0E0000000006181E008181000FC00FE00F40A7
:0200000400F00A
:1000000003010001017D87E0005B89982329FFFF40
:10001000FA00FA00FFFFFFFFFFFFFFFFFFFFFFFFF8
:100020000039A1E8003855E0006C3720006C37201B
:10003000FFFFFFFFFFFFFFFFFFFFFFFFFFFFFFFFD0
:10004000FFFFFFFFFFFFFFFFFFFFFFFFFFFFFFFFC0
:10005000FFFFFFFFFFFFFFFFFFFFFFFFFFFFFFFFB0
:1000600003030002FFFFFFFFFFFFFFFF005B93C0E2
:04007000005B8F742E
:00000001FF
